:020000020000FC
:100000000C942A000C943B000C943C000C943D0092
:100010000C943E000C943F000C9440000C94410062
:100020000C9442000C9443000C9444000C94450042
:100030000C9446000C9447000C9448000C94490022
:100040000C944A000C944B000C944C000C944D0002
:100050000C944E0004E00EBF0FE50DBF0FEF07BB81
:1000600000E607B907E806B9369A3699FECF05B11A
:10007000009508BBF9CF18951895189518951895FF
:100080001895189518951895189518951895189508
:0E0090001895189518951895189518951895A7
:00000001FF
